:1000000003C018951895189501E005BF02E009BFD7
:1000100000E808B900E001BD00E00BBF01E005BF4A
:100020000FEF07BBD02E112718BBF12E67E061BB85
:1000300062BB0AEF002E02E2102E09EB202E0BEA23
:10004000302E03E6402E0BEC502E0BED602E02EA14
:10005000702E0BEF802E0BEE902E22273327442795
:100060000FE0E02ECE2CBE2CAE2C8AE0AA2700C0DA
:100070005FEF06E003BF2A95F1F731503C3FD9F717
:100080003DE73A95F1F762BBEC2DF0E07081A030CE
:1000900009F0746078BB76E072BB00C02A95F1F776
:1000A00031503C3FD9F73DE73A95F1F762BBEB2D74
:1000B000F0E07081746078BB75E072BB00C02A9577
:1000C000F1F731503C3FD9F73DE73A95F1F762BB84
:1000D000EA2DF0E07081A03009F0746078BB73E025
:1000E00072BB413E19F04A9531F6C2CF3CE13A95D8
:1000F000F1F700E003BF08B701FF01C0AFEFAA2787
:1001000040EA99275527ECE0F0E0CE2CBE2CAE2C2F
:1001100002B7081718F0081B9395FBCF0083E15036
:10012000F040092F99270030A1F7EB3009F4008344
:0801300002BF02E008BF9FCFEF
:00000001FF
